:020000040800F2
:10000000E00C0020610200087B180008731800084B
:100010007718000899030008F11C00080000000090
:10002000000000000000000000000000A101000826
:100030009D03000800000000FD0100087D18000875
:100040008502000885020008850200088502000874
:100050008502000885020008850200088502000864
:100060008502000885020008850200088502000854
:100070008502000885020008850200088502000844
:100080008502000885020008850200088502000834
:100090008502000885020008850200088502000824
:1000A0008502000885020008850200088502000814
:1000B0008502000885020008850200088502000804
:1000C00085020008850200088502000885020008F4
:1000D00085020008A11C00088502000885020008AE
:1000E00085020008850200088502000885020008D4
:1000F00085020008850200088502000885020008C4
:1001000085020008850200088502000885020008B3
:1001100085020008850200088502000885020008A3
:100120008502000885020008850200088502000893
:1001300085020008A1030008850200088502000866
:100140008502000885020008850200088502000873
:100150008502000885020008850200088502000863
:100160008502000885020008850200088502000853
:1001700085020008850200088502000800000000D2
:100180008502000885020008DFF810D000F0F2F8C0
:100190000048004705250008AFF30080E00C002070
:1001A0002C4B19680868B0E8F04F80F30988BFF35A
:1001B0006F8F4FF0000080F311887047000000003F
:1001C00008480068006880F308884FF0000080F35A
:1001D000148862B661B6BFF34F8FBFF36F8F00DF35
:1001E00000BF00BF08ED00E0DFF80C00016841F43B
:1001F00070010160704700BF88ED00E0EFF30980F7
:10020000BFF36F8F134B1A681EF0100F08BF20ED5D
:10021000108A20E9F04F106009B44FF0500080F3CD
:100220001188BFF34F8FBFF36F8F02F063FC4FF065
:10023000000080F3118809BC19680868B0E8F04F25
:100240001EF0100F08BFB0EC108A80F30988BFF3CE
:100250006F8F704720000020EFF30580704700008B
:100260000948016841F47001016008488047084866
:100270000047FEE7FEE7FEE7FEE7FEE7FEE7FEE7F4
:10028000FEE7FEE7FEE7000088ED00E091180008B9
:10029000890100082DE9F05F0546002092469B4643
:1002A00088460646814640241BE02846414647468C
:1002B000224600F04FF853465A46C01A914110D3D7
:1002C00011461846224600F036F82D1A67EB010851
:1002D0004F4622460120002100F02DF817EB0009BF
:1002E0004E41201EA4F10104DFDC484631462A4677
:1002F0004346BDE8F09F10B5431A934209D28318D4
:10030000881803E010F8011D03F8011D521EF9D2F0
:1003100010BD40EA01039B0703D009E008C9121F82
:1003200008C0042AFAD203E011F8013B00F8013BAF
:10033000521EF9D210BD202A04DB203A00FA02F145
:10034000002070479140C2F1200320FA03F31943C3
:1003500090407047202A04DB203A21FA02F0002165
:10036000704721FA02F3D040C2F1200291400843C5
:1003700019467047064C074D06E0E06840F001035F
:1003800094E8070098471034AC42F6D3FFF700FF1B
:10039000C8310008E831000800BFFEE770470000E0
:1003A00010B50A49886A01F0ABFF08B102F092F873
:1003B0004FF480310548006800F5805041614021CC
:1003C0000248006800F58050416110BD9C0100208A
:1003D00010B5002201B909E0012901D10A0205E0A6
:1003E000022901D10A0201E04FF440720E4B1B6852
:1003F00023F440730C4C236023461B681343236093
:1004000023461B6823F0F803236023461B6802245D
:1004100044EAC0042343044C236023461B6843F48E
:100420008033236010BD0000103C02401C4800686F
:1004300000F40070B0B11A48006820F40070184948
:10044000086000BF0846006840F400600860084685
:10045000006820F40060086000BF0846006840F4AF
:10046000007008600E48006800F48060B0B10C486D
:10047000006820F480600A49086000BF08460068F0
:1004800040F4805008600846006820F480500860FE
:1004900000BF0846006840F48060086070470000B4
:1004A000003C02400A4A126822F44072084B1A606B
:1004B0001A46126842F004021A601A4612684FF493
:1004C000803343EA00231A43014B1A60704700004F
:1004D000103C0240074A126822F44072054B1A6031
:1004E0001A4612681A601A46126842F001021A602F
:1004F00001707047103C024010B50D49096821F4A5
:1005000040710B4C21602146096841F44071216023
:100510002146096841F001012160026000BF00BF6F
:1005200000BFBFF36F8F00BF00BF00BF436010BDAF
:10053000103C0240084A126822F44072064B1A60CE
:100540001A46126842F480721A601A46126842F023
:1005500001021A6001807047103C0240084A12688C
:1005600022F44072064B1A601A46126842F4007276
:100570001A601A46126842F001021A600160704760
:10058000103C02402348006800F0100040B12248AF
:10059000C06940F010002049C86110201D49086062
:1005A0001C48006800F0200040B11B48C06940F0C2
:1005B00008001949C86120201649086015480068DC
:1005C00000F0400040B11448C06940F004001249F6
:1005D000C86140200F4908600E48006800F08000A4
:1005E00040B10D48C06940F002000B49C86180204D
:1005F000084908600748006800F0020040B106485A
:10060000C06940F020000449C86102200149086027
:10061000704700000C3C02407C01002070B504468D
:10062000002500201449C86100F072FA054609E06F
:10063000601C38B124B100F06BFA401BA04201D914
:10064000032070BD0D48006800F480300028EFD111
:100650000A48006800F0010010B101200749086055
:100660000648006800F0F20018B1FFF78BFF012088
:10067000E7E70020E5E700007C0100200C3C024099
:1006800070B50446A56D00F043FA064694F83500AF
:10069000022808D08020606500BF002084F8340064
:1006A00000BF012070BD2068006820F0160021689E
:1006B00008602068406920F0800021684861206C53
:1006C00008B9A06C28B12068006820F008002168F3
:1006D00008602068006820F00100216808600FE0D1
:1006E00000F016FA801B05280AD92020606500BF9B
:1006F000002084F8340000BF032084F83500D1E7DF
:100700002068006800F001000028E9D194F85C102E
:100710003F208840A86000BF002084F8340000BF5C
:10072000012084F835000020BCE7014691F835002F
:10073000022803D08020486501207047052081F8F9
:1007400035000868006820F001000A681060002089
:10075000F3E700002DE9F04104460E46012700258D
:1007600000BF2548007E012802D10220BDE8F081AB
:1007700001202149087600BF4CF25030FFF74EFFB0
:100780000746002F31D1401E3060206801280FD16C
:10079000207C6168FFF786FE4CF25030FFF73EFF89
:1007A00007461648006820F00400144908601AE063
:1007B000A56812E0217C2846FFF70AFE4CF2503073
:1007C000FFF72CFF07460D48006820F0FA000B49A0
:1007D00008600FB1356005E06D1CD4E902100844D3
:1007E000A842E7D800BFFFF721FE00BF0020024962
:1007F000087600BF3846B9E77C010020103C024073
:100800000348006840F0004001490860002070473C
:10081000103C02402DE9F04106460F4614461D46A5
:100820004FF0010800BF1F48007E012802D10220BE
:10083000BDE8F08101201B49087600BF4CF2503022
:10084000FFF7ECFE8046B8F1000F23D126B9E1B2E4
:100850003846FFF73FFE12E0012E04D1A1B2384620
:10086000FFF768FE0BE0022E04D121463846FFF761
:1008700075FE04E022462B463846FFF73DFE4CF25B
:100880005030FFF7CBFE80460748006820F001009B
:100890000549086000BF00200249087600BF4046B5
:1008A000C6E700007C010020103C024000200949FE
:1008B000096801F0004159B10749064A0C3A116034
:1008C000064911600349096801F0004101B10120A6
:1008D00070470000103C024023016745AB89EFCD13
:1008E000F8B502460B460025002400200021DEE07A
:1008F000012606FA01F51E6806EA0504AC4275D128
:100900001E7906F00306012E04D01E7906F00306B8
:10091000022E13D190684F000326BE40B0434F0013
:10092000DE68BE4030439060506801268E40B04380
:100930001E79C6F300168E40304350601E7906F0D3
:100940000306032E09D0D0684F000326BE40B043F3
:100950004F009E68BE403043D0601E7906F003060B
:10096000022E13D1CF0802F1200656F827004E07B9
:10097000F70E0F26BE40B0434F07FF0E1E69BE4064
:100980003043CF0802F1200646F8270010684F00D8
:100990000326BE40B0431E7906F003064F00BE405A
:1009A000304310605E6806F08056B6F1805F7DD1FE
:1009B00000BF00260096404E366846F480463E4F03
:1009C0003E603E46366806F48046009600BF00BF93
:1009D0003A4E8F0856F827008E07370F0F26BE4075
:1009E000B043374EB24202D1002624E05EE0354EDD
:1009F000B24201D101261EE0334EB24201D102269D
:100A000019E0324EB24201D1032614E0304EB24218
:100A100001D104260FE02F4EB24201D105260AE093
:100A20002D4EB24201D1062605E02C4EB24201D134
:100A3000072600E008268F073F0FBE4030431F4EB9
:100A40008F0846F82700264E3068A0435E6806F4FB
:100A50008036B6F5803F00D12043214E3060361DF0
:100A60003068A0435E6806F40036B6F5003F00D15A
:100A700020431B4E361D3060361D3068A0435E6833
:100A800006F48016B6F5801F00D12043144E0836B8
:100A90003060361D3068A0435E6806F40016B6F577
:100AA000001F00D120430E4E0C363060491C102927
:100AB000FFF41EAFF8BD0000443802400838014082
:100AC000000002400004024000080240000C024006
:100AD000001002400014024000180240001C0240B6
:100AE000003C014010B5426921EA020302EA010418
:100AF00043EA0443836110BD0AB1816101E00B0444
:100B00008361704701480068000C7047002004E0D2
:100B1000014800687047000010000020034800688A
:100B20000349097808440149086070471000002013
:100B30001800002010B50D48006840F400700B4903
:100B400008600846006840F4806008600846006855
:100B500040F480700860032000F080F80F2000F05F
:100B600007F800F02BF8002010BD0000003C024008
:100B700070B504460E4800784FF47A71B1FBF0F07E
:100B80000C490968B1FBF0F5284600F01DFC08B1DE
:100B9000012070BD102C07D200222146501E00F00B
:100BA0001EF80548046001E00120F2E70020F0E7AC
:100BB00018000020000000201400002070470146AB
:100BC0000846002809DB00F01F0301229A40430970
:100BD0009B0003F1E023C3F8002100BF70472DE91B
:100BE000F05F80460D461646002701F093F8074651
:100BF00039462A46334601F00700C0F1070ABAF128
:100C0000040F02D94FF0040A01E0C0F1070AD146EF
:100C100000F1040ABAF1070F02D24FF0000A01E016
:100C2000A0F1030AD4464FF0010A0AFA09FAAAF120
:100C3000010A0AEA020A0AFA0CFA4FF0010B0BFA4F
:100C40000CFBABF1010B0BEA030B4AEA0B04214648
:100C5000404601F067F8BDE8F09F000000BF00F0DB
:100C60000702064B19684FF6FF031940044B0B436C
:100C700043EA0221014B196000BF70470CED00E010
:100C80000000FA0570B504460D460CB9012070BD90
:100C90005848006800F00700A84209D255490D7075
:100CA0000846006800F00700A84201D00120EEE7E6
:100CB000207800F0020002281DD1207800F0040006
:100CC000042805D14C48006840F4E0504A490860C7
:100CD000207800F00800082805D14748006840F453
:100CE0006040454908604448006820F0F000A16871
:100CF000084341490860207800F00100A8B360680B
:100D0000012807D13C4808380068C0F34040B8B912
:100D10000120BCE76068022802D06068032807D180
:100D2000354808380068C0F3406048B90120AEE794
:100D3000314808380068C0F3400008B90120A6E730
:100D40002D48006820F00300616808432A490860C4
:100D5000FFF7DEFE064609E0FFF7DAFE801B41F2F0
:100D60008831884202D9032091E707E022480068D1
:100D700000F00C006168B0EB810FEDD11D480068F8
:100D800000F00700A84209D91A490D70084600680A
:100D900000F00700A84201D0012078E7207800F099
:100DA0000400042807D11448006820F4E050E168EA
:100DB000084311490860207800F00800082808D18D
:100DC0000D48006820F46040216940EAC1000A49EA
:100DD000086000F03FF808490968C1F30311074AA9
:100DE000515CC8400649086006480068FFF7C0FE2D
:100DF00000204CE7003C02400838024068310008FF
:100E00000000002014000020014800687047000026
:100E10000000002000B5FFF7F7FF04490968C1F39F
:100E20008221034A515CC84000BD000008380240DE
:100E30007831000800B5FFF7E7FF04490968C1F3FE
:100E40004231034A515CC84000BD000008380240EE
:100E5000783100082DE9F047002400250026A1463E
:100E60002548006800F00C0020B1042805D00828AF
:100E70003AD105E0DFF8849039E0DFF8849036E07D
:100E80001D48001F006800F03F041B48001F006859
:100E900000F4800078B11A481749091F0968C1F3A6
:100EA0008811A0FB01700146224600233846FFF757
:100EB000F1F905460EE011480F49091F0968C1F311
:100EC0008811A0FB01700146224600233846FFF737
:100ED000E1F905460848001F0068C0F30140401CC6
:100EE0004600B5FBF6F902E0DFF8109000BF00BF46
:100EF0004846BDE8F0870000083802400024F400AE
:100F000000127A00F8B504460CB90120F8BD20782B
:100F100000F00100002874D0F948006800F00C00CF
:100F200004280DD0F648006800F00C00082813D102
:100F3000F348001F006800F48000B0F5800F0BD16B
:100F4000EF4808380068C0F34040002859D0606876
:100F5000002856D10120D9E700BF6068B0F5803F76
:100F600008D1E7480838006840F48030E44908397F
:100F700008601EE06068B0F5A02F0DD1E048083889
:100F8000006840F48020DE4908390860084600689F
:100F900040F4803008600CE0D9480838006820F43C
:100FA0008030D749083908600846006820F480205E
:100FB000086000BF606890B1FFF7AAFD054606E033
:100FC000FFF7A6FD401B642801D903209EE7CC480B
:100FD00008380068C0F340400028F1D011E0FFF766
:100FE00097FD054606E0FFF793FD401B642801D9F5
:100FF00003208BE7C24808380068C0F3404000284F
:10100000F1D1207800F0020002285FD1BC480068CE
:1010100000F00C0058B1BA48006800F00C00082835
:101020001CD1B748001F006800F48000B0B9B44874
:1010300008380068C0F3400020B1E068012801D002
:10104000012063E7AE480838006820F0F800216905
:1010500040EAC100AA490839086037E0E06800B3F7
:101060000120A8490860FFF753FD054606E0FFF799
:101070004FFD401B022801D9032047E7A04808384C
:101080000068C0F340000028F1D09D48083800688F
:1010900020F0F800216940EAC10099490839086048
:1010A00014E0002097490860FFF732FD054606E08E
:1010B000FFF72EFD401B022801D9032026E79048A8
:1010C00008380068C0F340000028F1D1207800F013
:1010D000080008282CD16069A8B101208A4908605D
:1010E000FFF716FD054606E0FFF712FD401B02283C
:1010F00001D903200AE782486C300068C0F3400041
:101100000028F1D014E000207F490860FFF700FDBF
:10111000054606E0FFF7FCFC401B022801D903202E
:10112000F4E677486C300068C0F340000028F1D145
:10113000207800F00400042870D10027704838306F
:10114000006800F0805090B900BF002000906C480B
:101150003830006840F080506949383108600846EE
:10116000006800F08050009000BF00BF0127674872
:10117000006800F48070B0B96448006840F4807082
:1011800062490860FFF7C4FC054606E0FFF7C0FCB3
:10119000401B022801D90320B8E65C48006800F42F
:1011A00080700028F2D000BFA068012808D1544800
:1011B0006830006840F001005149683108601DE066
:1011C000A06805280DD14E486830006840F0040042
:1011D0004B49683108600846006840F0010008602B
:1011E0000CE047486830006820F00100444968314D
:1011F00008600846006820F00400086000BFA0688E
:10120000A8B1FFF785FC054609E0FFF781FC401B0C
:1012100041F28831884202D9032077E626E0384837
:1012200068300068C0F340000028EED013E0FFF7FC
:101230006FFC054608E0FFF76BFC401B41F288316C
:10124000884201D9032061E62D4868300068C0F368
:1012500040000028EFD1012F07D12948383000681D
:1012600020F0805026493831086000BFA06900286E
:1012700045D02348006800F00C0008285DD0A06924
:10128000022845D100201F490866FFF741FC0546AA
:1012900006E0FFF73DFC401B022801D9032035E69C
:1012A000174808380068C0F340600028F1D1D4E93D
:1012B00007010843616A40EA81110122A06AC2EB7A
:1012C000500041EA00412C20005D41EA00600C49D9
:1012D000091F086001200B490866FFF719FC054645
:1012E00006E0FFF715FC401B022801D903200DE69C
:1012F000034808380068C0F340600028F1D049E096
:101300000838024000004742800E4742007000400B
:10131000002021490866FFF7FBFB054606E0FFF7C2
:10132000F7FB401B022801D90320EFE51B480068AA
:10133000C0F340600028F2D12CE0A069012800D160
:10134000E4E51648001D0668A069012820D006F4CF
:101350008001E06981421BD106F03F01206A814291
:1013600016D147F6C0703040616AB0EB811F0FD1D3
:1013700006F440310122A06AC2EB5000B1EB004FED
:1013800006D106F070612C20005DB1EB006F01D03A
:101390000120BBE50020B9E50000474200380240CB
:1013A000042808D14FF0E021096941F004014FF011
:1013B000E022116107E04FF0E021096921F004010A
:1013C0004FF0E0221161704770B504462546681E53
:1013D000B0F1807F01D301200FE0681E4FF0E021C3
:1013E00048610F214FF0FF3000F09CFC00204FF0CF
:1013F000E021886107200861002070BD70477047B8
:1014000001460022002391F83D2091F83E3042EA47
:10141000030070472DE9F84F0446206805682068EE
:10142000C668206847694FF00009CA4605F00F09F1
:10143000B9F1000F0AD105F0200038B106F0200004
:1014400020B1204600F063FABDE8F88FB9F1000F33
:1014500072D007F0010018B906F4907000286BD024
:1014600005F0010030B106F4807018B1206C40F036
:101470000100206405F0040030B107F0010018B14C
:10148000206C40F00200206405F0020030B107F04B
:10149000010018B1206C40F00400206405F0080041
:1014A00048B106F0200010B907F0010018B1206C17
:1014B00040F008002064206C70B305F0200028B1D3
:1014C00006F0200010B1204600F021FA20684069A3
:1014D000C0F3801A206C00F0080010B9BAF1000FB8
:1014E00023D0204600F0E8F92068406900F0400071
:1014F000402816D12068406920F0400021684861EA
:10150000A06B50B15648A16B0865A06BFFF70DF9B1
:1015100010B1A06B016D88470CE02046FFF76FFF0C
:1015200008E02046FFF76BFF04E02046FFF767FF67
:101530000020206488E7FFE7206B012879D105F0BF
:101540001000002875D006F01000002871D000BFF0
:10155000002000902068006800902068406800909B
:1015600000BF00BF2068406900F04000402839D12A
:10157000A06B006840681FFA80F8B8F1000F30D007
:10158000A08D40452DDDA4F82E80A06BC069B0F57C
:10159000807F1FD02068C06820F480702168C860F8
:1015A0002068406920F00100216848612068406996
:1015B00020F0400021684861202084F83E0000208F
:1015C00020632068C06820F010002168C860A06B0C
:1015D000FFF756F8A08DE28D801A81B22046FFF702
:1015E0000DFF31E7A08DE18D401A1FFA80F8E08DE4
:1015F000E8B1B8F1000F1AD02068C06820F49070EC
:101600002168C8602068406920F0010021684861B5
:10161000202084F83E00002020632068C06820F06D
:1016200010002168C86041462046FFF7E7FE0BE73F
:10163000FFE705F0800030B106F0800018B12046C9
:1016400000F0FDFA00E705F0400030B106F0400080
:1016500018B1204600F04BF9F6E600BFF4E60000B2
:10166000A518000810B504460CB9012010BDA069EA
:1016700000B100E000BF94F83D0028B9002084F8D4
:101680003C00204600F028F8242084F83D00206823
:10169000C06820F400502168C860204600F096F928
:1016A0002068006920F49040216808612068406942
:1016B00020F02A00216848612068C06840F400508A
:1016C0002168C86000202064202084F83D0084F850
:1016D0003E000020CAE7000010B586B004462E493F
:1016E0002068884255D100BF00BF002000902B48E1
:1016F000006840F01000294908600846006800F0C2
:101700001000009000BF00BF00BF00BF00BF00205E
:10171000009022481438006840F001001F49143935
:1017200008600846006800F00100009000BF00BF9C
:1017300000BF00BF00BF002000900846006840F0D6
:10174000010008600846006800F00100009000BF3A
:1017500000BF00BF481501900220029001200390B5
:10176000022004900720059001A90D48FFF7B8F862
:101770004FF4806001900720059001A90848FFF709
:10178000AFF82520FFF71BFA032211462520FFF7AB
:1017900026FA06B010BD0000001001404438024097
:1017A0000000024070B504460D46164694F83E000F
:1017B000202816D105B10EB9012070BD00BF94F8E4
:1017C0003C00012801D10220F7E7012084F83C0009
:1017D00000BF0020206332462946204600F00CFA64
:1017E000EBE70220E9E700001D4A0168914236D18B
:1017F0001C49098801F4004189BB1A49098801F490
:10180000804171B1184909780A2903D00021154A8D
:10181000118024E01349098841F40041114A1180E4
:101820001DE0114909780D2906D10E49098841F4B6
:1018300080410C4A118012E00B490978094A12884C
:10184000C2F30D02094B995406490988491C054AFF
:10185000118011460988C72901DD002111807047D8
:10186000001001400C0000200E000020700000203D
:10187000704700BFFEE700BFFEE7704710B5FFF7F7
:101880004DF901F03FFA012801D001F08FF910BDA8
:101890000348006840F47000014908607047000088
:1018A00088ED00E070B50546AC6B0020E085E08473
:1018B0002046FFF7A4FD70BD0168C96821F490714E
:1018C0000268D1600168496921F001010268516133
:1018D000016B012905D10168C96821F01001026876
:1018E000D160202180F83E1000210163704710B5BF
:1018F00004462068C06820F040002168C8602020AD
:1019000084F83D002046FFF7B3FF002010BD70B5FE
:10191000044694F83E00222856D1A068B0F5805FB6
:101920000CD1206950B90025A66A20684068C0F330
:1019300008003080A06A801CA06215E0A56A00261D
:10194000A068B0F5805F03D0A06828B9206918B9F5
:1019500020684068287004E02068406800F07F003C
:101960002870A06A401CA062E08D401E80B2E08515
:1019700040BB2068C06820F020002168C860206853
:10198000C06820F480702168C8602068406920F039
:10199000010021684861202084F83E00206B012866
:1019A0000AD12068C06820F010002168C860A18DAD
:1019B0002046FFF723FD02E02046FFF715FF002039
:1019C000206370BD0020FCE70220FAE72DE9F84F04
:1019D00004462068006920F44050E168084321680B
:1019E00008612169A068084361690843E169084307
:1019F00000902068C06849F20C6188430099084350
:101A00002168C8602068406920F44070A1690843DB
:101A10002168486176492068884203D0754920686A
:101A2000884203D1FFF706FA814602E0FFF7F2F998
:101A30008146E069B0F5004F6CD102206168A0FBDF
:101A4000015003461920A9FB007001462A4638467A
:101A5000FEF720FC6421B0FBF1F04FEA001A0220EF
:101A60006168A0FB01510B461920A9FB00712A46B1
:101A70003846FEF70FFC834602206168A0FB015048
:101A800003461920A9FB00712A463846FEF702FCDE
:101A90006421B0FBF1F000EBC00101EB0010ABEBF7
:101AA0008000322101EBC0006421B0FBF1F000F0B6
:101AB000F8000AEB400A02206168A0FB01500346CF
:101AC0001920A9FB007001462A463846FEF7E2FBC2
:101AD000834602206168A0FB015003461920A9FB40
:101AE00000712A463846FEF7D5FB6421B0FBF1F0C1
:101AF00000EBC00101EB0010ABEB8000322101EBE9
:101B0000C0006421B0FBF1F000F0070050442168F0
:101B100088606AE004206168A0FB01500346192038
:101B2000A9FB007001462A463846FEF7B3FB824601
:101B300004206168A0FB015003461920A9FB007036
:101B400001462A463846FEF7A5FB6421B0FBF1F0BA
:101B500000EBC00101EB0010AAEB8000322101EB89
:101B600000106421B0FBF1F000F0F00A042061687D
:101B7000A0FB017003461920A9FB00513A462846F4
:101B8000FEF788FB6421B0FBF1F00AEB001A042099
:101B90006168A0FB01510B461920A9FB00712A4680
:101BA0003846FEF777FB834604206168A0FB0150AE
:101BB00003461920A9FB007001462A463846FEF765
:101BC00069FB6421B0FBF1F000EBC00101EB0010F8
:101BD000ABEB8000322101EB00106421B0FBF1F08F
:101BE00000F00F00504421688860BDE8F88F0000C5
:101BF000001001400014014010B5034699629A8517
:101C0000DA8500201864222083F83E0000BF0020FF
:101C100083F83C0000BF1868C06840F480701C68FE
:101C2000E0601868406940F001001C686061186855
:101C3000C06840F020001C68E060002010BD014634
:101C400091F83D00212828D18868B0F5805F0BD13C
:101C5000086948B90A6A1088C0F308000B68586020
:101C6000086A801C086205E00B6A581C0862187834
:101C70000B685860C88C401E80B2C88458B9086888
:101C8000C06820F080000B68D8600868C06840F029
:101C900040000B68D860002070470220FCE700007D
:101CA00070B500240F4D1048FFF7B4FB00BF03E0F0
:101CB000641CAC4200D904E00B48FFF7A1FB2028CC
:101CC000F6D100BF002403E0641CAC4200D906E05A
:101CD000012206490448FFF765FD0028F4D100BF42
:101CE00070BD0000FFFF0100380100200E00002041
:101CF00000BFFEE70FB4054B10B503A9044A0298D4
:101D000000F034F810BC5DF814FB00002523000837
:101D10000800002002480068C0F30220704700005D
:101D20000CED00E010B5002804DB0A07130E054A8D
:101D3000135406E00A07140E034A00F00F031B1F9A
:101D4000D45410BD00E400E018ED00E002E008C843
:101D5000121F08C1002AFAD170477047002001E025
:101D600001C1121F002AFBD1704700002DE9FF4F6F
:101D70008DB00F460546002606E025280BD0DDE98C
:101D80000F1290476D1C761C28780028F5D111B0F1
:101D90003046BDE8F08F0024A246A1460122E94961
:101DA00000E0044315F8013F203B02FA03F008422B
:101DB000F7D128782A2810D06FF02F022878A0F1C8
:101DC0003001092914D80AEB8A0102EB410144F0E1
:101DD000020400EB010A6D1CF0E701CF5FEA000A84
:101DE00003D544F40054CAF1000A44F002046D1C07
:101DF00028782E2817D115F8010F44F004042A285A
:101E00000ED06FF02F022878A0F1300109290AD8EE
:101E100009EB890102EB410100EB01096D1CF2E7BE
:101E200057F8049B6D1C28786C280FD006DC4C28D2
:101E300017D068280DD06A2814D104E0742810D077
:101E40007A280FD10DE044F400140AE044F4801421
:101E500001E044F440146978814202D104F5801411
:101E60006D1C6D1C28786E281ED00CDC632830D0C9
:101E700004DC00288BD0582811D19FE0642867D05B
:101E800069280CD164E073282DD004DC6F2872D04F
:101E9000702804D194E075286ED078286DD0DDE9E3
:101EA0000F129047761C4BE1C4F30250022806D073
:101EB000032809D0042801CF09D0066040E101CFF2
:101EC000F117C0E900613BE101CF068038E10670FF
:101ED00036E117F8040B8DF8000000208DF80100A2
:101EE000EB46012003E057F804BB4FF0FF306107D9
:101EF0004FF0000102D40DE008F101018846494588
:101F00000FDA8045F8DB1BF808100029F4D108E04F
:101F100008F1010188468142FADB1BF8081000290C
:101F2000F6D1DDE90F23AAEB08008146214600F037
:101F300031F9304400EB080604E0DDE90F121BF82C
:101F4000010B9047B8F10108F7D221464846F2E06C
:101F50000A21C4F302524FF0000B0891022A04D068
:101F600001CFC117032A09D00AE0FF1D27F0070798
:101F7000F7E8020108E02CE01EE01FE000B2C11704
:101F8000042A01D140B2C117021E71F1000206DA23
:101F90000023D0EB030063EB01012D2202E02205B8
:101FA00004D52B228DF82420012203E0E20701D082
:101FB0002022F7E7904653E00A210BE0102109E0C8
:101FC00010214FF0000B44F004044FF00809089171
:101FD00003E008214FF0000B0891C4F30252022ADB
:101FE00004D001CF0021032A06D006E0FF1D27F010
:101FF0000707F7E8020103E080B2042A00D1C0B26B
:102000004FF0000822072BD52A78702A07D0DDF878
:1020100020C08CF0100C5CEA0B0C05D00EE04022C6
:102020008DF82420012208E050EA010306D0302375
:102030008DF824308DF8252002229046089B83F0ED
:10204000080353EA0B030BD150EA010201D16207E6
:1020500006D530228DF824204FF00108A9F101099E
:102060002A78582A04D038A20B9208AA0A920BE0C8
:102070003AA2F9E75B46089AFEF70CF90B9B9B5CCA
:102080000A9A521E0A92137050EA0102F2D10A987B
:10209000ADEB000000F1200B600702D524F4803482
:1020A00001E04FF00109D94502DDA9EB0B0000E08A
:1020B000002000EB0B0141440890AAEB010AE00369
:1020C00006D4DDE90F232146504600F063F80644AC
:1020D0004FF0000908E009A911F80900DDE90F1225
:1020E000904709F10109761CC145F4DBE0030CD5EA
:1020F000DDE90F232146504600F04CF8064404E089
:10210000DDE90F1230209047761C0899481E089090
:102110000029F5DC08E00A980A990078491C0A9120
:10212000DDE90F129047761CBBF10001ABF1010B0A
:10213000F1DC21465046DDE90F2300F019F8064492
:102140006D1C21E609280100303132333435363731
:1021500038396162636465660000000030313233F3
:102160003435363738394142434445460000000093
:102170002DE9F041044600251E461746880404D484
:1021800005E039462020B0476D1C641EF9D528466D
:10219000BDE8F0812DE9F041044600251E46904639
:1021A000C80301D5302700E02027880404D505E0C6
:1021B00041463846B0476D1C641EF9D52846BDE837
:1021C000F081000000B587B01848194988601948A7
:1021D000C8606FF07F40086142F2F56048610020FE
:1021E0004860012008600622134800F005FB062223
:1021F00001A9114800F0ECFA10A00399FFF77AFD4D
:1022000013A00499FFF776FD16A00599FFF772FD5C
:102210001AA00699FFF76EFD1EA00299FFF76AFD4E
:1022200024A00199FFF766FD07B000BDC0A8010A10
:10223000C8040020C0A8010100000108434F4E4619
:102240004947493A69703A25640D0A0A00000000BE
:10225000434F4E464947493A67773A25640D0A0A83
:1022600000000000434F4E464947493A6E65746D81
:1022700061736B3A25640D0A0A000000434F4E4615
:102280004947493A6C6F63616C706F72743A2564A8
:102290000D0A0A00434F4E464947493A6F6274613E
:1022A000696E696E675F69705F6D6F64653A25641A
:1022B0000D0A0A00434F4E464947493A6D61736B18
:1022C0003A25640D0A0A000070B504460420FFF7A1
:1022D00067F80A48046025464FF47A7045434FF08A
:1022E000E020006940F002004FF0E021086108465C
:1022F0004561006940F00100086170BD04000020E4
:10230000014600200A6802F0004252B90A6802F44D
:10231000004232B90A6802F4807212B10A68C2F34C
:102320000D40704700BF054A126802F04002002AC3
:10233000F9D0C2B2014B5A60704700000010014052
:1023400000B587B000BF00BF00200190384800688A
:1023500040F01000364908600846006800F01000A0
:10236000019000BF00BF00BF00BF00BF0020019070
:102370000846006840F0100008600846006800F059
:102380001000019000BF00BF00BF00BF00BF0020D1
:1023900001900846006840F0100008600846006898
:1023A00000F01000019000BF00BF00BF00BF00BFE1
:1023B000002001900846006840F0010008600846CF
:1023C000006800F00100019000BF00BF00BF1020B6
:1023D000029000200390012004900220059002A9A1
:1023E0001448FEF77DFA0820029000200390012097
:1023F00004900220059002A90E48FEF771FA04200D
:10240000029000200390012004900220059002A970
:102410000848FEF765FA0120029000200390022090
:102420000490059002A90448FEF75AFA07B000BDCF
:1024300030380240001002400000024000B587B072
:1024400000BF00BF002001902048006840F020003D
:102450001E4908600846006800F02000019000BF97
:1024600000BF00BF00BF00BF002001900846006809
:1024700040F0200008600846006800F0200001904D
:1024800000BF00BF00BF48150290012003900490D8
:102490000220059002A90E48FEF722FA4FF4806050
:1024A000029002A90A48FEF71BFA00BF012251025E
:1024B0000748FEF721FB00BF00BF0122910204483C
:1024C000FEF71AFB00BF07B000BD00003038024025
:1024D0000014024008B569460848006800F080FB17
:1024E00000BF009838B14FF0805005490860BFF335
:1024F0004F8FBFF36F8F00BF08BD00001C0000208E
:1025000004ED00E008B5FEF715FB00BF00200090C9
:102510001148006840F008000F490860084600684C
:1025200000F00800009000BF00BF0723022208212E
:102530004FF4A87000F0D2F9A820FFF7C5FE4FF4C1
:10254000E13000F031FAFFF779FFFFF7F9FE00F014
:1025500047FA002008BD00003038024010B5084896
:10256000006800F0ADF9B0F5967F08D9FEF7D0FA13
:10257000034908604FF480610248FEF7B3FA10BDCA
:102580006C000020001402402DE9F04104460F4683
:1025900015464FF00008A66B206C48B9206800284B
:1025A0002CD1A06800F0B2FC80460020A06025E09D
:1025B0007DB93946226C6068FDF79DFE216C60682C
:1025C00008446060D4E90101884217D32068606044
:1025D00014E03946226CE068FDF78DFE216CE0685E
:1025E000411AE1602168E068884203D2216CA0684A
:1025F000411AE160022D01D106B1761E701CA06364
:102600004046BDE8F0810000F1B50098846C0026DA
:102610002CB940F6D53220A128A0FFF76BFBA06BA8
:10262000E16B884201D2012000E0002028B940F689
:10263000D63219A121A0FFF75DFBA06BE16B8842A8
:1026400027D294F94550002269462046FFF79CFFA7
:102650000646681C60B9606A08B9012000E00020E5
:10266000B0B904F1240000F0D9FC88B101260FE0D4
:102670007F2D01D0012000E0002028B940F6F6327D
:1026800005A10EA0FFF736FB681C40B284F8450098
:1026900000BF3046F8BD00002E2E5C2E2E5C4D692A
:1026A00064646C6577617265735C467265655254EB
:1026B0004F535C71756575652E6300004572726FCE
:1026C000723A2025732C2025640D0A000948006801
:1026D000006808B9012000E0002020B14FF0FF3071
:1026E0000549086005E003480068C06800680249C1
:1026F0000860704724000020500000200246B2F11C
:10270000006F05D302F0030010B9B2F1016F01D9D7
:1027100000207047B1F1006F05D301F0030010B93C
:10272000B1F1016F01D90020F3E70120F1E70000CA
:1027300001461C48814201D2002070471A4881425C
:1027400001D20120F9E71948814201D20220F4E7C1
:102750001748814201D20320EFE71648814201D297
:102760000420EAE71448814201D20520E5E7134836
:10277000814201D20620E0E71148814201D20720C0
:10278000DBE71048814201D20820D6E70E4881429B
:1027900001D20920D1E70D48814201D20A20CCE7BD
:1027A0000B20CAE7004000080080000800C00008B5
:1027B00000000108000002080000040800000608EC
:1027C0000000080800000A0800000C0800000E08BD
:1027D00030B503460C461546002206E0184600F0C8
:1027E00007F844F822001B1D521CAA42F6D330BD44
:1027F00001460868704700002DE9F04387B00446A1
:102800000E4617464FF000090025A846002001900B
:10281000254604EB870841462846FFF76FFFFEF781
:1028200045F82548006820F4806023490860234863
:1028300085421DD219E02846FFF7DAFF401C78B127
:10284000002002902846FFF773FF049001200590B6
:102850000220069001A902A8FDF77CFF08B106E05E
:102860002D1D4CF25030FDF7D9FE4545E3D300BF96
:102870004CF25030FDF7D2FE8146B9F1000F0FD176
:102880000BE0D6F800C06246002321460220FDF787
:10289000C1FF00B103E0241D361D4445F1D300BF44
:1028A0000548006840F4806003490860FDF7A8FF10
:1028B00007B0BDE8F0830000003C02400000FF1FAD
:1028C00070B50446FEF724F90546A54201D3281B3E
:1028D00070BDC4F1FF302844FAE700002DE9F04153
:1028E00092B080460C4615461E46002700BF0020C9
:1028F00000902A48006840F0805028490860084647
:10290000006800F08050009000BF00BF00BF0020B2
:1029100000902348006840F4804021490860084640
:10292000006800F48040009000BF00BF01200190CB
:10293000000402900220079041050891CDF82880FC
:1029400009940B950C9601A8FEF7DCFA07461FB117
:10295000012012B0BDE8F0810F200D9002200E90F2
:1029600000200F904FF4A05010904FF48050119021
:1029700004210DA8FEF786F907460FB10120E8E70C
:10298000FEF7C0F841F20101884205D10548006810
:1029900040F48070034908600020DAE740380240C4
:1029A00000700040003C024010B5044609480A4946
:1029B00008600846446000218160C1600161816156
:1029C0000C214161FEF74EFE012204490248FEF748
:1029D000E9FE10BD00100140380100200E0000206B
:1029E0000648FFF787F90122114605A0FFF782F993
:1029F000FFF7E8FB01E0FFF7B1FDFCE780310008DD
:102A0000555345525F4D41494E493A766572736957
:102A10006F6E2025642E25640A00000001460A69B5
:102A2000D1E901309860D1E90103586050688842CB
:102A300001D188685060002008611068401E106055
:102A40001068704770B5FDF707FC0546102D11D3CF
:102A500005F1E02090F8F04310480078844201DB53
:102A6000012000E0002028B940F217320CA11BA081
:102A7000FFF740F91D48006800F4E0601C49096850
:102A8000884201D8012000E0002028B940F2273216
:102A900003A112A0FFF72EF970BD00006400002012
:102AA0002E2E5C2E2E5C4D6964646C6577617265B8
:102AB000735C4672656552544F535C706F727461FB
:102AC000626C655C525644535C41524D5F434D34D9
:102AD000465C706F72742E63000000004572726F66
:102AE000723A2025732C2025640D0A000CED00E0BD
:102AF0006800002010B51B48006818B101201A4971
:102B000008602DE000201849086018480068B0FAF5
:102B100080F0C0F11F0404EB8400154951F8200037
:102B200008B1012000E0002028B940F6024211A1BE
:102B300019A0FFF7DFF804EB84010D4A02EB8100D6
:102B400041684968416000F1080142688A4202D147
:102B50004168496841604168C968134A116000BF13
:102B600010BD00005C000020440000203800002060
:102B7000E40100202E2E5C2E2E5C4D6964646C6591
:102B800077617265735C4672656552544F535C742D
:102B900061736B732E6300004572726F723A202569
:102BA000732C2025640D0A002000002010B500BF02
:102BB000502080F31188BFF34F8FBFF36F8F00BF9A
:102BC00000F0B0F818B14FF080500449086000BF21
:102BD000002080F3118800BF10BD000004ED00E06C
:102BE0002DE9F04707460D463C462CB940F2AD4270
:102BF00037A140A0FFF77EF8206C08B9012000E063
:102C0000002028B940F2B14231A13AA0FFF772F892
:102C1000206808B9A06808B9012000E0002028B9A0
:102C200040F2B6422AA133A0FFF764F8FFF70AFF8B
:102C300000BF5021EFF3118081F31188BFF34F8F54
:102C4000BFF36F8F00BF0646D4F838A0E06B504545
:102C500035D994F945900AF10100A06309F101000A
:102C6000C0B9A06C38B12046FFF7CEFC20B31DB32D
:102C70000120286020E0606A08B9012000E00020FF
:102C8000D0B904F1240000F0C9F9A8B1A5B1012020
:102C9000286011E0B9F17F0F01D0012000E0002091
:102CA00028B940F235520AA112A0FFF723F809F122
:102CB000010040B284F845004FF0010801E04FF0F8
:102CC000000800BF86F3118800BF4046BDE8F087CA
:102CD0002E2E5C2E2E5C4D6964646C657761726586
:102CE000735C4672656552544F535C7175657565CA
:102CF0002E6300004572726F723A2025732C2025D6
:102D0000640D0A000549096809B9012005E0044974
:102D1000096809B9022000E0002070473C0000204B
:102D20005C0000202DE9F0414FF000085F4800688A
:102D300000287DD15E480068451C5D480560002D77
:102D40001DD15C480068006808B9012000E000203F
:102D500028B940F6C72258A160A0FEF7CBFF55481E
:102D60000768624800685349086060480760604827
:102D70000068401C5E490860FFF7A8FC00BF5D4882
:102D80000068854277D300BF4A480068006808B9E8
:102D9000012000E0002020B14FF0FF3055490860CD
:102DA00068E044480068C068C4686668B54202D2FA
:102DB000504806605EE06069D4E902128A60D4E996
:102DC00002214A60211D42688A4201D1E1684160C6
:102DD000002262610168491E0160A06A98B1A06A80
:102DE000D4E907128A60D4E907214A6004F1180186
:102DF00042688A4201D1216A41600022A2620168D0
:102E0000491E016000BF94F82C10012088403A4907
:102E10000968084338490860E16A01EB8101374AD3
:102E200002EB81014868A0608268E260211D00E039
:102E300033E0826851608160E16A01EB81012F4AD1
:102E400002EB81026261E16A01EB81012B4A52F8D7
:102E50002110491CE26A02EB8202284B43F822103F
:102E60002749E06A0968C96A88428DD34FF0010892
:102E70008AE700E000BF22480068C06A00EB8000DB
:102E80001E4951F82000012801D94FF001081D48C2
:102E9000006808B14FF0010804E01B480068401CBE
:102EA000194908604046BDE8F08100005C00002040
:102EB00034000020240000202E2E5C2E2E5C4D6954
:102EC00064646C6577617265735C467265655254C3
:102ED0004F535C7461736B732E6300004572726FA5
:102EE000723A2025732C2025640D0A00280000204A
:102EF000480000205000002038000020E40100209D
:102F000020000020440000204000002070B505464D
:102F10002C460026002D5ED030480068844201D146
:102F2000012000E0002028B941F24F022CA135A079
:102F3000FEF7E0FE206D28B941F2500228A131A031
:102F4000FEF7D8FE206D401E2065E16CE06A8842E5
:102F500041D0206D00283ED1201DFFF75FFD40B914
:102F600094F82C10012088402A4909688143294897
:102F70000160E06CE062E06AC0F12000A06194F8BA
:102F80002C10012088402349096808432149086022
:102F9000E16A01EB8101204A02EB81014868A060EF
:102FA0008268E260211D826851608160E16A01EB04
:102FB0008101194A02EB81026261E16A01EB810140
:102FC000154A52F82110491CE26A02EB8202124BA8
:102FD00043F822100126304670BD0000200000207A
:102FE0002E2E5C2E2E5C4D6964646C657761726573
:102FF000735C4672656552544F535C7461736B73B6
:103000002E6300004572726F723A2025732C2025C2
:10301000640D0A0038000020E401002070B5064667
:10302000F068C4682CB940F682423CA144A0FEF787
:1030300061FEA06AD4E907128A60D4E907214A60D8
:1030400004F1180142688A4201D1216A41600022DC
:10305000A2620168491E01603D48006800283DD118
:103060006069D4E902128A60D4E902214A60211D14
:1030700042688A4201D1E1684160002262610168D0
:10308000491E016094F82C100120884031490968DC
:10309000084330490860E16A01EB81012E4A02EBE6
:1030A00081014868A0608268E260211D82685160E9
:1030B0008160E16A01EB8101274A02EB81026261D2
:1030C000E16A01EB8101244A52F82110491CE26AAD
:1030D00002EB8202204B43F8221010E01F4948689F
:1030E000E0618268226204F11801826851608160A7
:1030F0001A4AA26211460968491C116000BF1849AA
:10310000E06A0968C96A884204D901250120154985
:10311000086000E00025284670BD00002E2E5C2EC1
:103120002E5C4D6964646C6577617265735C467290
:10313000656552544F535C7461736B732E6300006A
:103140004572726F723A2025732C2025640D0A0097
:103150005C00002038000020E40100208C040020E6
:1031600020000020440000200000000000000000BB
:10317000010203040607080900000000010203041D
:10318000555345525F4D41494E493A3D3D3D3D3DC8
:103190003D3D3D3D3D3D3D3D3D65746865726E651F
:1031A000745F736F756E645F616371756973697461
:1031B000696F6E5F636172643D3D3D3D3D3D3D3DE8
:1031C0003D3D3D3D3D0A0000E83100080000002083
:1031D000700000004C1D00085832000870000020EC
:1031E000700C00005C1D00080024F40000000000CA
:1031F00000000000000000000000000010000000BF
:1032000001000000000000000000000000000000BD
:1032100000000000000000000000000000000000AE
:10322000000000000000000000000000000000009E
:10323000000000000000000000000000000000008E
:103240001F00000000000000AAAAAAAA00000000B7
:08325000000000000000000076
:040000050800018965
:00000001FF
